:020000040800F2
:1000000020060020C90000086D080008D507000878
:1000100000000000000000000000000000000000E0
:10002000000000000000000000000000D5000008F3
:100030000000000000000000D7000008CD0F0008FD
:10004000DB00000800000000B10C0008DB00000825
:10005000DB0000083D0500083F050008DB00000844
:1000600000000000DB000008DB000008DB000008E7
:10007000DB000008DB000008DB00000800000000D7
:10008000DB0000080000000000000000DB000008AA
:10009000DB000008DB000008DB000008DB000008D4
:1000A000DB000008DB000008DB000008411200084C
:1000B000491200080348854600F016F90048004739
:1000C000211F0008200600200448804704480047FC
:1000D000FEE7FEE7FEE7FEE7FEE7FEE7E10F0008CA
:1000E000B500000830B50B4601460020202201244F
:1000F00009E00D46D5409D4205D31D469540491B5C
:100100002546954040191546521E002DF1DC30BDA4
:1001100003460B439B0703D009E008C9121F08C020
:10012000042AFAD203E00B780370401C491C521ECB
:10013000F9D27047D2B201E00270401C491EFBD2D6
:1001400070470022F6E710B513460A4604461946E2
:10015000FFF7F0FF204610BD30B505462A460B4696
:1001600010781C78521C5B1C002801D0A042F7D0EC
:10017000002C03D0002802D06D1CEFE7284630BDCC
:10018000421C0178401C0029FBD1801A704710B531
:10019000002200E0521C835C8C5CA34201D1002B46
:1001A000F8D1D8B2E1B2401A10BD30B504460020F3
:1001B000034600E05B1C934203D2E05CCD5C401B35
:1001C000F8D030BD03460A780270401C491C002A52
:1001D000F9D1184670470321001D401E0378120212
:1001E0001A43491EF9D5104670470346032208708A
:1001F000000A491C521EFAD51846704770B50646CB
:1002000001F0DEF9046805460A220021304600F0BC
:1002100033F82C6070BDF0B51FB40646002082B0E4
:1002200005464024019100901BE0019922460F46AB
:10023000304600F07BF8049A059B801A994110D350
:1002400010461946224600F061F8361A8F41019790
:10025000224601200021009F00F058F838184D4137
:1002600000902046641E0028DFDC019B0098294690
:10027000324607B0F0BD0000F7B5009C0F460026DF
:100280002578641C002D05D000F062F80068405D00
:10029000C007F5D12B2D02D02D2D18D0641E394664
:1002A0002046029A00F058F8002F04D03968A14285
:1002B00001D1009939607105022400290BDA40420E
:1002C000002803DD01F07CF90460A007FEBD0120D9
:1002D00080020643E3E70028F8DA01F071F90460D0
:1002E0000048FEBDFFFFFF7F064C0125064E05E0DE
:1002F000E36807CC2B430C3C98471034B442F7D347
:10030000FFF7DCFE182400083824000810B5202A66
:1003100004DB0146203A9140002010BD914020238B
:100320009C1A0346E3401943904010BD10B5202AA3
:1003300004DB0846203AD040002110BD0B46D340D4
:10034000D0402024A21A91400843194610BD000055
:1003500000487047D8220008F7B582B0029C0027F9
:100360002078641C15460197302802D0002D15D046
:1003700015E020780127641C782804D0582802D082
:10038000002D09D00BE0002D01D0102D07D1002742
:1003900010252078641C02E0082500E00A250026CC
:1003A000009610E00099012769430818020C2946BD
:1003B00080B2714300908E183804864201D3012028
:1003C00001902078641C294600F019F80028E9DA29
:1003D0000398002805D0002F01D0641E00E0029C85
:1003E00004600198002806D001F0EAF802210160BB
:1003F000C81E05B0F0BD009930040843F9E73A285B
:1004000000D23038202302469A43412A01D31046B5
:100410003738884201D30020C0437047FEB52F20F3
:100420000121400400F07AFB0024684604718471C5
:1004300003254571C471022609206946C00600964D
:1004400000F027F901276846077184714571C6716C
:100450003003009009206946C00600F01AF968468A
:10046000077184714571C47120200090092069468C
:10047000C00600F00EF94020009009206946C00631
:1004800000F007F91020009009206946C00600F02E
:1004900000F98020009009206946C00600F0F9F8B4
:1004A0000420009009206946C00600F0F2F80820F8
:1004B000009009206946C00600F0EBF80920F02101
:1004C000C00600F037F9FEBD70B5074D040008D036
:1004D000012C05D1002205A1002000F059FD2C704F
:1004E00070BD002209A1F7E718000020446562757D
:1004F0006720434F4D2073656C63657420746F20D3
:100500004D6F64656D210D0A000000004465627541
:100510006720434F4D2073656C63657420746F20B2
:100520004D4355210D0A000001B5034800990160B3
:1005300001680029FCD108BD000000207047704709
:10054000F0B5072410A312A20021CD17AD0F6D182E
:10055000AD08AD004D1B2D182E785F5C491C7E4008
:100560002E70A142F1DB0C230021CC17A40F6418DC
:10057000A408A4000C1B24182578565C491C75405F
:1005800025709942F1DBF0BD50432D544F4F4C0084
:1005900050432D544553542D544F4F4C00000000F0
:1005A0000149C8607047000000200240F0B50B27E9
:1005B00006463F04384600F05BF804280FD1084C8B
:1005C0002069022528432061666120694021084393
:1005D0002061384600F04CF82169A9432161F0BD43
:1005E0000020024008490420CA68D20701D0012037
:1005F0007047CA68D20601D502207047C96849070A
:10060000FBD503207047000000200240024801692A
:10061000802211430161704700200240F0B50B2792
:1006200006463F040D46384600F022F804280CD157
:10063000064C20690121084320613580384600F0CE
:1006400017F82169490849002161F0BD00200240E6
:1006500004480169090603D5034941600349416023
:10066000704700000020024023016745AB89EFCDB1
:1006700000B50346FFF7B6FF02E0FFF7B3FF5B1ECE
:10068000012803D0002B00D1052000BD002BF4D1A0
:10069000FAE7F0B50022012423460D6893401D407F
:1006A0009D422AD10D79012D01D0022D12D18768EA
:1006B00055000326AE40B74387604E79AE4085684B
:1006C0002E43866085889D43858085888B799340FD
:1006D0001D438580066855000323AB409E4306609A
:1006E0000E790768AE403E430660C6689E43C6600A
:1006F000CB79AB40C5682B43C360521C102ACBD3C7
:10070000F0BD4B07DB0E9A40C90810B589000818E8
:10071000016A0F249C40A1430162016A11430162F6
:1007200010BD0246128A00200A4200D00120704704
:100730000185704781617047F7B50646002500784E
:1007400086B02C462B4600281CD00A786846002A22
:1007500018D007E0C2545B1C3D2A13D03B2A11D0AD
:10076000491C641C0A78002A01D0142CF2DB3D21BC
:1007700001550027641C075501463046FFF7ECFC85
:10078000001909E0002009B0F0BD089A401C117062
:100790000899491C6D1C08910178202903D93B292F
:1007A00001D0282DF1DB089807702846EBE7000000
:1007B00010B500280BD00022054B8900D04202D092
:1007C0005C58A45C8454521CD2B20C2AF6D310BDDF
:1007D0002C000020FEE7000010B504460121C802ED
:1007E00000F0A8F95D2000F049FA002801D000F0DF
:1007F000B9F9074800F02AF8062000F01BF8204657
:1008000000F01EF800F00EF800F004F810BD000033
:10081000555500000249014808607047CCCC0000E3
:10082000003000400249014808607047AAAA000051
:10083000003000400149486070470000003000402F
:10084000014988607047000000300040014908609D
:10085000704700000030004008B51B216846017059
:1008600001214170817000F003F808BD704700005D
:1008700030B5837801210278002B15D094080E4BF7
:10088000A400E41823689207D50EFF22AA409343E0
:1008900042789207120EAA401A4322600078C006DE
:1008A000C00E8140054804E0D006C00E81400348D8
:1008B0008030016030BD000000E400E000E100E0B5
:1008C000F0B595B005461C223C490DA8FFF720FC69
:1008D00000210DA88A008258491C1278002AF9D1FB
:1008E0000024491E07E0A2008258EB1C16E01F7886
:1008F000BE4211D0641C8C42F5DB8C421AD001221E
:100900002FA1002000F044FB314E230000F04AFEEE
:10091000060A1428313D4C12521C5B1C1678002E1E
:10092000E5D1EAE700222BA1104600F031FB0120BF
:10093000FFF7CAFD15B0F0BD6A4629A12846FFF7AA
:10094000FBFE6846FFF75AFCC3B2F37326A23221BE
:10095000684600F011FE694626A000F0FDFD20E08B
:10096000F37B25A23221684600F006FE694621A0ED
:1009700020E026A23221684600F0FEFD01226946F1
:10098000002000F005FB01200AE023A23221684686
:1009900000F0F2FD01226946002000F0F9FA002083
:1009A000307400F011FAC5E70948817A407A0902EB
:1009B00001431CA000F0D0FDBCE70000302000087F
:1009C000554152542053544152543333333333003E
:1009D0006C00002047542B544D3A4F4B0D0A000039
:1009E0004144445200000000414444523D3D3D25F5
:1009F000640D0A002573000052542B5241444452A6
:100A00003A414444523D25640D0A000052542B5390
:100A1000444542554700000052542B534E4F444525
:100A20004255470052543530315F5625640D0A0057
:100A3000FEB5C5782C4E0446014630462A1F01F00B
:100A40005BF96219203A517F127F0902274D511834
:100A50002279EB7B89B29A4202D0012224A109E0DB
:100A6000814202D0012225A104E0A078032805D00C
:100A7000012225A1002000F08BFAFEBD00F070F9E4
:100A8000AA2269460A70BB224A7003228A700B228E
:100A9000CA70EA7B0A71EE224A71887107223046D9
:100AA00001F02AF96946C871000A0872DD2048720F
:100AB00055208872012676030920C0068661154DEF
:100AC00000246F46395D284600F064FC402128462A
:100AD00000F0CCFB0028F9D0641CE4B20B2CF1D35D
:100AE0000D480681FEBD0000FFFF00006C000020E5
:100AF00061646472206572726F000000435243208B
:100B00006572726F00000000636D64206572726F21
:100B1000720000000038014020000048044A00290B
:100B2000516901D0014300E08143516170470000E9
:100B300000100240044A0029D16901D0014300E0BD
:100B40008143D1617047000000100240044A00292F
:100B5000916901D0014300E0814391617047000039
:100B6000001002400348416A01221206114341620B
:100B70007047000000100240014610B52F204004CD
:100B8000FFF7CCFF10BD0000F8B5354D044668688E
:100B90000C21344E084004D0334A042803D00828DE
:100BA00003D0266014E0226012E0696868680123BF
:100BB00089021B040F0F1840BF1C00281CD0E86AD4
:100BC0000107090F1046491CFFF78CFA7843206093
:100BD0006868264B0006000F1A5C20680146D14069
:100BE00061606A685205520F9A5CD140A1602A6B1D
:100BF000D20505D41E4A09E01E4847432760E7E7AF
:100C00006A68520401D44A0800E08A08E2602A6B4C
:100C10005306194A03D4184B1233236100E02261B2
:100C20002B6BDB0601D4666100E060612B6B9B07D8
:100C30000FD0296B8907890F01290CD0286B8007F9
:100C4000800F022809D0286BC043800700D1A6611D
:100C5000F8BDA161F8BDA061F8BDA261F8BD0000BA
:100C60000010024000127A00001BB700550000205F
:100C7000809FD50000093D00008000000346002051
:100C80000A495A090CD0012A0CD0022A0CD0496B0F
:100C9000DA06D20E012393400B4200D001207047A8
:100CA0000968F5E7096AF3E7496AF1E700100240CD
:100CB000704730B500231C4607E005192D88CD5438
:100CC0002D0A5B1CCD545B1CA41C9442F5D330BD93
:100CD000F8B511221B491C48FFF7EBFF194C002601
:100CE00020786927651C482805D118A1601CFFF7EA
:100CF0004EFA002818D0012216A1002000F048F971
:100D000011211048FFF71DFA482020700FA1601C28
:100D1000FFF758FA2F72380A0A4968720B3100201F
:100D2000FFF763FAE67308E0687A297A000208435D
:100D3000692805D02F72380A6872267400F044F8CA
:100D4000F8BD00006C000020003C00085254353013
:100D50003153000052737420506172610000000032
:100D6000F8B5002404260925ED06AE6115480827CC
:100D700007810120FFF7D8FBAF610320FFF7D4FB09
:100D800002212846FFF7CDFC012800D101240027CD
:100D90006006040E0B4806810120FFF7C5FBAE611B
:100DA0000120FFF7C1FB02212846FFF7BAFC01280A
:100DB00000D104437F1CFFB2072FE9D3014806810D
:100DC0002046F8BD2000004810B506482024846164
:100DD00011220549054800F053FB024820300481E8
:100DE00010BD0000000400486C000020003C00081A
:100DF00030B504468DB000200390E57801222146ED
:100E000000F0C6F80D2221462748FFF7CEF900284A
:100E100023D00D2221462448FFF77AF92A1F2146C4
:100E2000224800F069FF014660192038427F007FA8
:100E30001202801880B2884204D11D492079C97BF2
:100E4000884202D001221BA104E0A078062806D027
:100E500001221DA1002000F09BF80DB030BD012241
:100E60001CA1002000F094F8002003A92218527958
:100E70000A54401CC0B20428F8D36846C27B817B68
:100E8000407B6B4607C36846037B15A21E2104A85E
:100E900000F072FB012204A9002000F079F803A9F8
:100EA000042000F016FBD8E710020020FFFF00002E
:100EB0006C000020637263206F722061646472654D
:100EC00072726F0D0A000000636D64206572726FAC
:100ED0000D0A0000736574206C656420000000003A
:100EE000253032782E2E253032782E2E253032784D
:100EF0002E2E2530327800001CB5002122480191A9
:100F00000091026801231B041A4302605B00052262
:100F1000120204681C400094019C641C0194009C13
:100F2000002C02D1019C9442F3D10268920328D58F
:100F300001210091154A1121116041684160416809
:100F4000416041683F221204914341604168092297
:100F5000120411434160016801221206114301602D
:100F600001688901FCD541688908890041604168B0
:100F700002221143416041680907890F0229FAD111
:100F80001CBD00911CBD000000100240002002406A
:100F900070B514460D46012812D00A48007C00287E
:100FA0000ED00846FFF7ECF80104090C08D02846DB
:100FB00000F0F4F9002C03D0022103A000F0EEF9B8
:100FC00070BD00006C0000200D0A0000034801689D
:100FD000002902D00168491E01607047000000200E
:100FE00010B5144801680122114301604168124A9A
:100FF000114041600168114A1140016001680122FD
:1010000092049143016041683F2212049143416080
:10101000C16A09090901C162016BFF22543291437F
:101020000163416B49084900416300218160FFF77A
:1010300063FF10BD001002400CB8FFF8FFFFF6FE82
:10104000F0B5734C734F87B02146384600F015F960
:10105000002828D0384600F099F9694608700978C8
:10106000384600F097F92146384600F0F0F86A4E0D
:1010700000257078317800020843684C002801D0C0
:10108000E58033E068460178E0883218401C83B27E
:10109000D1706348E3800078012813D0F078892864
:1010A00077D0E580F57008215E4800F0DFF8012870
:1010B00006D1384600F06AF90821384600F0C5F834
:1010C00007B0F0BD032B69D9F078AA2804D0CC284A
:1010D0001FD052284BD05DE03079BB285AD1042B69
:1010E00006D0A078834206D9E580A570F570E7E7C1
:1010F00068460078A070E078DD2853D16846007813
:1011000055284FD13370180A7070F018C570E580FB
:101110004FE03079DD283DD101206070042B13D0E1
:10112000A1788B4213D900913FA2142101A800F0AD
:1011300023FA012201A90020FFF72AFFE580A5700C
:10114000F57003206070BBE768460078A070E07817
:10115000DD2827D168460078552823D13370180A36
:101160007070F018C570E5800220607021E0307961
:1011700054280FD1E0780D2814D1684600780A2849
:1011800010D13370180A7070F018C570E580A57022
:101190000FE030E0E580A570F5700AE0012B0CD07F
:1011A000022B1BD0C72B04D3E580A5703570280A0D
:1011B000707068460078E07075E768460078AA2885
:1011C000F7D068460078CC28F3D0684600785228DB
:1011D000EFD0684600784128DCD1EAE7684600781D
:1011E000BB28E6D068460078DD28E2D06846007863
:1011F0005428CFD1DDE7032BDED37079C01C0090DB
:101200008342D9D33370180A7070E5804BE7000031
:1012100005010500003801407D0000201800002075
:101220005400002000440040727863743D3D256402
:101230002C6D61786C656E3D3D3D25640D0A0000A6
:1012400010B5FFF7FDFE10BD7047016270470A0C34
:1012500001219140016270470029016802D00122FA
:10126000114301E049084900016070470246D26914
:1012700000200A4200D00120704730B50A04130E46
:101280000122144600258C40012B0ED0022B0ED0DB
:101290008368090C2340C0698A401040002B02D0AB
:1012A000002800D00125284630BD0368F1E74368D7
:1012B000EFE710B50B041C0E01238B40022C02D06B
:1012C000032C02D002E0001D00E008300168002A73
:1012D00001D0194300E09943016010BD70B5044688
:1012E000006888B00D464008400020606168032017
:1012F00000038143A8680843606021682148EA68C8
:101300000140686810432A690A4310432060A068BE
:1013100003210902884369690143A1606846FFF718
:1013200033FC1948844201D1069800E002982168F4
:101330000904296801D5490000E0890019225043B9
:10134000FEF7D0FE05466421FEF7CCFE060130090B
:10135000642148432168281A090407D5C000642184
:101360003230FEF7BFFE4007400F06E00001642167
:101370003230FEF7B7FE0007000F3043A08108B0FF
:1013800070BD0000F3E9FFFF00380140808CC0050C
:10139000C00D7047C905C90D01857047F3B5012718
:1013A0007F03092081B0C0060E46876100240A4DE4
:1013B0000CE00198015D2846FFF7ECFF402128462C
:1013C000FFF754FF0028F9D0641CA4B2B442F0D354
:1013D00002480781FEBD000000380140200000489F
:1013E00030B5012189B08803FFF7B0FB0921CD0694
:1013F00001222846FFF785F901220A212846FFF736
:1014000080F90320400206900220694608770320F5
:10141000487700248C770120C87706A92846FFF773
:1014200038F9E1204002059400900C20104D049002
:1014300001940294039469462846FFF74FFF012266
:101440000C492846FFF735FF01212846FFF704FF26
:1014500040212846FFF7F9FE0748C8218470C01CC8
:10146000FEF76FFE05496814088109B030BD000021
:1014700000380140050105007D00002020000048E3
:10148000F8B517460E460546FFF7E2F83420FFF799
:1014900087F81F20C006012128180904884217D2A6
:1014A000A80515D12846FFF781F8042810D100249B
:1014B0000AE030194078315D0002401881B22819E5
:1014C000FFF7ACF8A41CA4B2BC42F2D3FFF79EF81D
:1014D000F8BDF8B506460F4609201021C006FFF7F3
:1014E00027F929E03C7811200443002509204021F8
:1014F000C006FFF71DF9200605D509208021C0068A
:10150000FFF718F904E009208021C006FFF710F961
:101510000120FFF709F809204021C006FFF70AF96A
:101520000120FFF701F860066D1C040EEDB2082DD6
:10153000DCD3761EF6B27F1C002ED3D10924E4063C
:1015400010212046FFF7F6F80220FEF7EDFF1021EC
:101550002046FFF7EDF8F8BD0FB410B503A9044B12
:10156000044A029800F040F810BC08BC04B01847C8
:10157000FD1E0008200000200FB41CB50A46521EB4
:101580000192009007A9064B6A46069800F02CF8D5
:10159000009A002111701CBC08BC04B01847000060
:1015A0005D1A000830B47446641E2578641CAB4292
:1015B00000D21D46635D5B00E31830BC1847000095
:1015C000004870476800002002E008C8121F08C1E8
:1015D000002AFAD170477047002001E001C1121FB4
:1015E000002AFBD170470000FFB591B00F460546B9
:1015F000002606E025280AD0149A139990476D1CFE
:10160000761C28780028F5D1304615B0F0BD0024AE
:1016100000940121F34A029400E004436D1C2B78EE
:101620000846203B98401042F7D128782A280ED04F
:10163000022128780246303A092A15D8009A0A234E
:101640005A43303A80180C436D1C0090F1E701CFEB
:101650000090002805DA012040030443009840422E
:101660000090022004436D1C28782E2815D10420F8
:10167000044368786D1C2A280AD101CF6D1C0290A2
:101680000BE002990A225143303940186D1C029038
:101690002878014630390929F3D928786C2810D0E8
:1016A00006DC4C281AD068280ED06A2817D104E02E
:1016B000742813D07A2812D110E001204005044389
:1016C0000CE00121090501E0032109050C436978BB
:1016D000814203D10120000524186D1C6D1C28785F
:1016E00003906E281ED00CDC632831D004DC002867
:1016F0008AD0582811D1B2E064287BD069280CD157
:1017000078E073282DD004DC6F2870D0702804D1C5
:10171000A7E075286CD078286BD0149A139990475D
:10172000761C62E06002400F022807D003280AD02E
:10173000042838680AD006603F1D56E03868F11763
:1017400006604160F8E738680680F5E70670F3E761
:101750003878694608740020487404A80390012072
:1017600003E0386803900020C0433F1D61070FD598
:10177000002101E00199491C029A0191914213DA7A
:101780008142F7DB019A0399895C0029F2D10BE0D1
:10179000002101E00199491C01918142FADB019A83
:1017A0000399895C0029F5D101990098139A401A90
:1017B00000902146149B00F03BF9019980194618CE
:1017C00007E0039803990078491C0391149A139930
:1017D00090470198401E0190401CF2D12146149B75
:1017E000139A009800F014F986196D1C09E741E07E
:1017F00033E034E00A200021049005916002410F9B
:10180000022905D001CFC2179446032905D007E06D
:10181000FF1DFF08FF0003CF06E000B2C217944689
:10182000042902D140B2C1178C460022614694457A
:1018300006DA0A460021404291418C462D2102E001
:10184000210504D52B216A461176012103E0E10729
:1018500001D02021F7E7019154E00A200BE010208D
:1018600009E0102004900021042004430820059181
:10187000029003E008200021059104906002410FCE
:10188000022905D001CF00229446032906D006E0A4
:10189000FF1DFF08FF0003CF8C4603E080B2042940
:1018A00000D1C0B20021019121072BD503997029E5
:1018B00006D0049A1021059B4A401A4305D00EE039
:1018C00040216A461176012108E06146014306D0B5
:1018D00030216A4611760399517602210191049ACA
:1018E0000821059B4A401A430CD16146014301D1AE
:1018F000610707D530216A461176012101910299CD
:10190000491E02910399582904D037A103910FA9C8
:101910000F910DE039A1F9E76146059B049AFEF7A6
:101920007AFC039B8C469B5C0F9A521E0F9213709D
:1019300061460143F0D10F9807A9081A203003909F
:10194000600704D5012000048443029801E00120CF
:1019500002900399884201DD401A00E000204118FE
:101960000290019809180098401A0090E00306D4EC
:101970002146149B139A009800F05AF8861900200B
:10198000049008E006A9085C149A139990470498FB
:10199000401C761C049001998842F3DBE0030CD5CF
:1019A0002146149B139A009800F042F8861904E02F
:1019B000149A302013999047761C0299481E029081
:1019C0000029F5DC08E00F980F990078491C0F9169
:1019D000149A13999047761C0399481E0390002986
:1019E000F1DCFBE60928010030313233343536377B
:1019F000383961626364656600000000303132335B
:101A000034353637383941424344454600000000FA
:101A1000F8B5044600251E461746880404D405E0A0
:101A200039462020B0476D1C641EF9D52846F8BD04
:101A3000FFB50446002581B01E46C80301D53027F6
:101A400000E02027880404D505E038460399B04714
:101A50006D1C641EF9D5284605B0F0BD4A68002A01
:101A600006D00A68531C0B6010704868401E48601E
:101A700070470000F0B50024AFB025462746214648
:101A80000EA8FEF795FE0C2146A0FFF765FD0EAEF1
:101A9000315D46A0FFF760FD641C0C2CF8D345A017
:101AA000FFF75AFD0C210EA800F0E4F901462C9036
:101AB00041A0FFF751FD0EAB07CB002613AB47C388
:101AC0001796189641A116A81996FEF77BFB1A9651
:101AD0001B961C963FA11AA81D96FEF773FB414E5C
:101AE0002046384304D100221146302000F09EF8F1
:101AF000641CB44204D3002F01D16D1CEDB200244C
:101B0000032D1BD8FEF78EFE374841780278090274
:101B10001143E5D0C01CC9B26B462C9A00F004F901
:101B2000002806D004281ED0052820D0062820D062
:101B300024E00C220EA9352000F078F83522694601
:101B40002A48FFF7B6F807A80330FEF744FB2C99A4
:101B5000884218D108A8C1782548017025A0FFF750
:101B6000FBFC2FB0F0BD0C220EA9372004E00127AA
:101B700004E02C2213A9342000F058F81A49002060
:101B800008704870ACE7FEF74DFE641CB442FAD30F
:101B90001CA0FFF7E1FCFEF745FEFEF743FE022422
:101BA000F1E7000049445B25645D3A002530327856
:101BB000000000000D0A0000656E636F64655661E9
:101BC0006C75653A253038780D0A000050432D5465
:101BD0004F4F4C0050432D544553542D544F4F4CB0
:101BE00000000000C0C62D007D0000200038000865
:101BF00024000020536C6176654E756D3D3D3D259A
:101C0000640D0A00706C65617365207472792061DF
:101C10007574682D2D2D2D2D2D2D2D2D2D2D2D2D2A
:101C20002D2D2D2D2D2D0D0A00000000F0B5A1B099
:101C300001ABDF1CD41CE5B289266C4626716071AD
:101C40002648A5714088060AE67120720524002006
:101C500005E00E5C1E55641C401CE4B2C0B290420C
:101C6000F7D3E91C6846017001794170417900267B
:101C700081706D1E0CE003213046FEF733FA684692
:101C8000405CB95D484086214840B855761CF6B2A4
:101C9000AE42F0DB0021084601AD03E02A5C514072
:101CA000401CC0B2A042F9D32955641CE6B23146AB
:101CB0002846FFF773FB314609A0FFF74DFC0024CF
:101CC00005E0295D09A0FFF747FC641CE4B2B442BB
:101CD000F7D308A0FFF740FC21B0F0BD240000209E
:101CE00073656E645B25645D3A00000025303278D0
:101CF000000000000D0A000030B515460C46002318
:101D000004E02178641C00F005F85B1CAB42F8D3BA
:101D100030BD0000020A484000060249C00D085AC2
:101D20005040704754200008FFB5054687B0C01CDE
:101D300000902C7800221E46892C02D001200BB086
:101D4000F0BDA878C01C884201D00220F7E700202F
:101D50004B1E03E02F5C7A40401CC0B29842F9DB76
:101D60006F1838462038C07F904201D00320E6E744
:101D70006846017344736978817300240EE003217F
:101D80002046FEF7AFF903A8405C0099095D484082
:101D90008621484000990855641CE4B26878401ECA
:101DA000A042ECDC6878312804D0322804D03628F0
:101DB00049D103E00520C2E70620C0E7009CA41C2F
:101DC0002046FEF7BDFB207801026078084301023F
:101DD000A0780843E178000201430491217923208F
:101DE000815531461F31241D0498FEF7FEF900206D
:101DF0002178AA79641C51403154A74200D82C465E
:101E0000401CC0B21F28F3D3002021782A79641C1B
:101E10005140321820321171A74200D82C46401C84
:101E2000C0B21128F1D3352231460848FFF728FB0C
:101E300007A0099A0499FFF78FFB09990498884233
:101E400001D100207BE7042079E70000003800087A
:101E50006E657741757468496E666F3A25303878DB
:101E60002C746172676574636F64653A25303878E5
:101E70000D0A000030B5D1B00C460546FF220132F4
:101E80001D4910A8FEF744F900221346694604E0F4
:101E9000E85CC85442405B1CDBB2A342F8D362400A
:101EA00010AB9D5C002007E00A5C6A400546554087
:101EB0000D549D5C401CC0B2A042F5D300204200EE
:101EC0008318CA5C5B185C789B78624053400B5463
:101ED000401CC0B20428F2D308780102684640785A
:101EE0000843010268468078084301026846C078CA
:101EF00051B0084330BD00000C23000870B5074DF9
:101F00000446C1B22846FFF745FA40212846FFF7AC
:101F1000ADF90028F9D0204670BD0000003801401E
:101F20008AB0002501200895FEF726FE33487D2162
:101F3000C9000068FEF7D6F8314988420DD808403C
:101F40003049401E4861304B0722D8690002000A20
:101F50004C042043D8618D610A61FEF75FFAFFF7F8
:101F60003FFAFEF779FCFF20F530FEF735FCFEF76F
:101F7000AFFE692325A21E216846FFF7FDFA6946D8
:101F800028A0FFF7E9FA284C2570FFF773FD012020
:101F9000207008A90420FFF79CFA244CFEF742FCAD
:101FA0006078217800020843F8D0E178AA2905D0AA
:101FB0002046CC2909D052290ED016E02079BB2822
:101FC00013D1E01CFEF734FD0FE00179DD290CD1BF
:101FD000E01CFEF70DFF08E00179542905D1417995
:101FE0002B2902D1E01CFEF76BFCC821E01CFEF798
:101FF000A8F82570280A6070D0E7000004000020CF
:10200000FFFFFF0000E000E004ED00E05254353037
:1020100031532025642061707020676F2020676F26
:1020200020676F0025730000540000207D00002011
:10203000E4220008F0220008E8220008DC22000860
:1020400000230008F82200080823000810270000D9
:10205000020000000000C1C081C1400101C3C003F3
:10206000800241C201C6C006800741C70005C1C544
:1020700081C4400401CCC00C800D41CD000FC1CF04
:1020800081CE400E000AC1CA81CB400B01C9C009F4
:10209000800841C801D8C018801941D9001BC1DB94
:1020A00081DA401A001EC1DE81DF401F01DDC01D44
:1020B000801C41DC0014C1D481D5401501D7C01764
:1020C000801641D601D2C012801341D30011C1D174
:1020D00081D0401001F0C030803141F10033C1F3B4
:1020E00081F240320036C1F681F7403701F5C03544
:1020F000803441F4003CC1FC81FD403D01FFC03F04
:10210000803E41FE01FAC03A803B41FB0039C1F9F3
:1021100081F840380028C1E881E9402901EBC02B53
:10212000802A41EA01EEC02E802F41EF002DC1ED43
:1021300081EC402C01E4C024802541E50027C1E763
:1021400081E640260022C1E281E3402301E1C02173
:10215000802041E001A0C060806141A10063C1A373
:1021600081A240620066C1A681A7406701A5C06543
:10217000806441A4006CC1AC81AD406D01AFC06F03
:10218000806E41AE01AAC06A806B41AB0069C1A9F3
:1021900081A840680078C1B881B9407901BBC07B93
:1021A000807A41BA01BEC07E807F41BF007DC1BD43
:1021B00081BC407C01B4C074807541B50077C1B763
:1021C00081B640760072C1B281B3407301B1C07173
:1021D000807041B00050C190819140510193C05333
:1021E000805241920196C056805741970055C19543
:1021F00081944054019CC05C805D419D005FC19F03
:10220000819E405E005AC19A819B405B0199C059F2
:10221000805841980188C04880494189004BC18B52
:10222000818A404A004EC18E818F404F018DC04D42
:10223000804C418C0044C184818540450187C04762
:10224000804641860182C042804341830041C18172
:10225000818040400040404040404040404041413B
:10226000414141404040404040404040404040406B
:102270004040404040050202020202020202020205
:102280000202020202202020202020202020200202
:102290000202020202029090909090901010101092
:1022A000101010101010101010101010101010102E
:1022B00002020202020288888888888808080808C2
:1022C000080808080808080808080808080808088E
:1022D0000202020240000000552200085344454219
:1022E00055470000544D0000524144445200000044
:1022F0005341444452000000535645520000000030
:10230000534E4F4445425500000000006859636435
:10231000C8CCAAA7A2ABA56E6A568A57F4BBFEFA30
:1023200026212D290D093E3A37320A07F7F2FBF52F
:10233000FFF61C181314F1FDF90C9F089A97929B55
:10234000959F121B152C2823F92A2722242E672556
:102350002F98FC75F8F33C3833340304050F06015D
:102360007A7772626B83848EC4CB8782353F364F17
:102370003D399C989394424F4641818D4D49717DE2
:102380007996919D99C3C41DCECA7F767C7873746B
:102390007E7B751E1A171F16111D47195DC7C2CB0C
:1023A000C5CFD1DDD94C48C6C1CD61C9D78CFD8818
:1023B000A1ADA9B1BDB98B858F4B4586DCD8D3D4EF
:1023C000DED2DBD5DFD643444E4AE747ACA8A3A410
:1023D000AEBA0DB7B2AFA6E4EEEAE7E2E1ED0FE97F
:1023E00066616D69BBB5BFB6ECE80BE3525C656F27
:1023F0005853540C5E5B555F312F9A0B0B5A2B9E32
:102400000289593B0E516CEBDAE631F6D8B5B402CD
:10241000A8B8B402C0112000382400080000002031
:102420006C000000C8150008A42400086C000020FF
:10243000B4050000D815000800000000006CDC02A4
:102440000000000000000000010203040607080964
:10245000000000000000000000000000000000007C
:1024600000000000ACF7FF1FE8F7FF1F107AFF1F06
:10247000ACF7FF1F107AFF1F20F4F01F5000F81F69
:102480005000F81F9075FF1F20F4F01F000000009F
:10249000000102030401020304060708090000000A
:0424A0000000000038
:04000005080000B53A
:00000001FF
